S0100000636667315F6F75742E73726563FC
S3150800000010000020A10000089300000893000008D3
S315080000109300000893000008930000080000000001
S315080000200000000000000000000000009300000827
S3150800003093000008000000009300000893000008E1
S31508000040000000000000000000000000000004009E
S315080000500000000000000000000000000000000092
S315080000600120C046002801D0C046C0460020C04630
S31508000070C04600F000F800F001B834120746C04642
S31508000080C046C046C046C046C046384600F002F8DC
S31508000090FBE7FEE701491820ABBEFBE72600020096
S315080000A0C046C046C046C046FFF7DAFF7856341247
S315080000B00800000000000000FF000000000000002B
S315080000C000000000000000007F00000000000000A3
S315080000D0FF7F000000000000FFFFFF7F0000000018
S315080000E0FFFFFF7F00000000000000000000000086
S315080000F001000000000000000000000000000000F1
S3150800010002000000000000000100000000000000DE
S3150800011002000000000000000200000000000000CD
S3150800012004000000000000000200000000000000BB
S3150800013002000000000000000100000000000000AE
S31508000140020000000000000001000000000000009E
S315080001501000000000000000010000000000000080
S315080001601000000000000000010000000000000070
S315080001701000000000000000010000000000000060
S315080001801000000000000000FFFFFFFF0000000055
S31508000190FFFFFF7F00000000F1FFFFFFFFFFFFFFEB
S315080001A00000000000000000000000000000000041
S315080001B00000000000000000000000000000000031
S315080001C0000000000000000002000000000000001F
S315080001D00000000000000000000000000000000011
S315080001E000000000000000000800000000000000F9
S315080001F001000000000000000100000000000000EF
S3150800020008000000000000000100000000000000D7
S3150800021004000000000000000100000000000000CB
S3150800022004000000000000000400000000000000B8
S3150800023004000000000000000400000000000000A8
S315080002400400000000000000040000000000000098
S315080002500400000000000000040000000000000088
S315080002600400000000000000040000000000000078
S315080002700400000000000000040000000000000068
S315080002802000000000000000000000000000000040
S315080002900400000000000000080000000000000044
S315080002A00C00000000000000100000000000000024
S315080002B01400000000000000180000000000000004
S315080002C01C000000000000000C00000000000000F8
S315080002D0000000000000000004000000000000000C
S315080002E008000000000000000400000000000000F4
S315080002F008000000000000000000000000000000E8
S3150800030004000000000000000C00000000000000CF
S3150800031000000000000000000400000000000000CB
S3150800032008000000000000001000000000000000A7
S3150800033000000000000000000400000000000000AB
S3150800034008000000000000000C000000000000008B
S315080003500800000000000000000000000000000087
S315080003600400000000000000140000000000000067
S31508000370000000000000000004000000000000006B
S3150800038008000000000000000C000000000000004B
S31508000390100000000000000014000000000000002B
S315080003A0000000000000000004000000000000003B
S315080003B008000000000000000C000000000000001B
S315080003C010000000000000000C0000000000000003
S315080003D0000000000000000004000000000000000B
S315080003E008000000000000000C00000000000000EB
S315080003F000000000000000000400000000000000EB
S3150800040008000000000000000C00000000000000CA
S3150800041000000000000000000400000000000000CA
S3150800042008000000000000000C00000000000000AA
S3150800043000000000000000000400000000000000AA
S3150800044008000000000000004C000000000000004A
S31508000450F1FFFFFFFFFFFFFF0400000000000000A0
S315080004602000000000000000080000000000000056
S315080004701000000000000000180000000000000046
S315080004801C00000000000000000000000000000042
S31508000490000000000000000001000000000000004D
S315080004A0000000000000000002000000000000003C
S315080004B00F0000000000000000000000000000001F
S315080004C003000000000000000F000000000000000C
S315080004D00100000000000000FAFFFFFFFFFFFFFF1A
S315080004E004000000000000000000000000000000FA
S315080004F005000000000000000000000000000000E9
S3150800050006000000000000000000000000000000D7
S3150800051007000000000000000000000000000000C6
S315080005203500000000000000010000000000000087
S315080005300800000000000000350000000000000070
S315080005400100000000000000FDFFFFFFFFFFFFFFA6
S315080005500900000000000000000000000000000084
S315080005600A00000000000000010000000000000072
S31508000570000000000000000001000000000000006C
S315080005800B00000000000000010000000000000051
S31508000590010000000000000001000000000000004B
S315080005A01200000000000000020000000000000029
S315080005B00300000000000000000400000000000026
S315080005C0130000000000000000000000000000000A
S315080005D014000000000000000000000000000000F9
S315080005E00A000000000000000004000000000000EF
S315080005F015000000000000000000000000000000D8
S315080006000A000000000000000004000000000000CE
S3150800061016000000000000000000000000000000B6
S315080006200A000000000000000004000000000000AE
S315080006301700000000000000020000000000000093
S315080006400500000000000000000400000000000093
S315080006501800000000000000000000000000000074
S315080006601900000000000000000000000000000063
S315080006701A00000000000000000000000000000052
S315080006801B00000000000000000000000000000041
S31508000690D007000000000000000000000000000075
S315080006A01C00000000000000000000000000000020
S315080006B01D00000000000000060000000000000009
S315080006C00000000000000000785634120800000000
S315080006D004000000704770470120704712000000B0
S705080000A151
